:100000000C9434000C9449000C9449000C94490061
:100010000C9449000C9449000C9449000C9449003C
:100020000C9449000C9449000C9449000C9449002C
:100030000C9449000C9449000C9449000C9449001C
:100040000C9449000C9449000C9449000C9449000C
:100050000C9449000C9449000C9449000C944900FC
:100060000C9449000C94490011241FBECFEFD4E03A
:10007000DEBFCDBF11E0A0E0B1E0E2E8F1E002C0F8
:1000800005900D92A230B107D9F70E94AB000C94F5
:10009000BF000C9400008AB1806E8AB98091000183
:1000A00081FF03C08BB18F7102C08BB1806E8BB9A1
:1000B00008958093000108950C944B00982F80912F
:1000C00000014BB121E030E0B90102C0660F771F9B
:1000D0009A95E2F781FF04C0CB018095842302C08A
:1000E000CB01842B8BB90895982F809100014BB1DF
:1000F00021E030E0B90102C0660F771F9A95E2F760
:1001000081FF03C0CB01842B03C0CB0180958423E6
:100110008BB90895CF93C82F0E9474008FE19EE49D
:100120000197F1F700C000008C2F0E945E009FEF46
:100130002AE683E0915020408040E1F700C00000B3
:10014000CF91089585E00E948A0086E00E948A008F
:1001500087E00C948A0081E00E9459000E945C00B4
:100160000E94A20085E00E948A002FEF89E698E1B4
:10017000215080409040E1F700C00000F3CFF89498
:02018000FFCFAF
:0201820001007A
:00000001FF
